:100000000C9495020C94D9020C94D9020C94D90248
:100010000C94D9020C94D9020C94D9020C94D902F4
:100020000C94D9020C94D9020C941E0D0C94E20C81
:100030000C943D1B0C94D9020C94D9020C94D90257
:100040000C94D9020C94D9020C94D9020C94D902C4
:100050000C94D9020C94C31B0C94D9020C94D902B1
:100060000C94D9020C94D9020C94D9020C94D902A4
:100070000C94D9020C94D9020C94D9020C94D90294
:100080000C94D9020C94D9020C94D9020C94D90284
:100090000C94D9020C94D9020C94D9020C94D90274
:1000A0000C94D9020C94D9020C94D902260227028E
:1000B0002F0230022B7100001E00140004001D747A
:1000C000360219011F001A0016001B0037022C729D
:1000D00020000800070006003102287821001500E2
:1000E0000900190024020601220017000A00050079
:1000F0000000378134022A0000003800000036007A
:1001000016014C000000330000004A0023001C00D0
:100110000B00110000004D81240018000D0010009C
:100120002E00520025000C000E0034002E0228780C
:10013000260012000F001E022D002C722700130053
:100140002D023802250251002F0030001C011D0134
:100150000154000029002B000100010001000000F3
:100160003A000A300B300100E30001003B000C3084
:100170000D300100E20001003C0010300F300E3065
:10018000010001003D001130123013300100010068
:100190003E0014301530163000000100350001001B
:1001A0000000310000001B01B20001000000350218
:1001B000000001003F001730183019300000010026
:1001C00040000100010001004B000100410001005E
:1001D000010001004E004F0042000100010001003B
:1001E00049005000430001000100010046000100E9
:1001F0004400450001000100010000000000F0A1E2
:1002000001E1012602260127022702E10133023320
:10021000000111021101080208011A021A012C0240
:100220002C00013802380138023801E101170217A9
:1002300001120212010702070112021202E1012C4F
:10024000022C000105020501150215010802080132
:10025000040204010E020E013302330001110211E7
:1002600001180218010F020F010F020F0001150201
:1002700015010802080117021701180218011502DA
:1002800015011102110001090209010F020F0112EB
:1002900002120104020401170217012C022C0001B2
:1002A0000C020C0111021101170217012C022C0083
:1002B000010502050112021201120212010F020FC2
:1002C000012C022C0001160216011702170115025B
:1002D00015010C020C01110211010A020A012C0283
:1002E0002C00011902190104020401150215012C48
:1002F000022C000119021901120212010C020C0158
:10030000070207012C022C0001060206011202124C
:10031000011102110116021601170217012C022CFD
:100320000001160216011702170104020401170248
:1003300017010C020C01060206012C022C0001130D
:10034000021301150215010C020C01190219010416
:1003500002040117021701080208012C022C0001F7
:100360001302130118021801050205010F020F0103
:100370000C020C01060206012C022C0005010906E4
:10038000A101050719E029E7150025019508750168
:100390008102950175088101050819012905950556
:1003A000750191029501750391010507190029FF57
:1003B000150025FF950675088100C005010902A1F9
:1003C000010901A10005091901290515002501955B
:1003D0000575018102950175038101050109300947
:1003E000311581257F95027508810609381581250B
:1003F0007F950175088106050C0A38021581257F55
:10040000950175088106C0C005010980A10185021A
:1004100016010026B7001A01002AB70075109501D1
:100420008100C0050C0901A1018503160100269C6D
:10043000021A01002A9C02751095018100C0050175
:100440000906A101050719E029E71500250195080E
:1004500075018102050819012905950575019102AB
:1004600095017503910105071900297715002501EC
:10047000957875018102C01201100100000008ED9D
:10048000FE071301000102000109026D00040100D2
:10049000A0FA090400000103010100092111010073
:1004A00001223F000705810308000A090401000139
:1004B00003010200092111010001224D00070582FC
:1004C0000308000A090402000103000000092111C9
:1004D0000100012236000705830308000A0904030E
:1004E0000001030000000921110100012239000769
:1004F000058403100001040309041603450072007B
:1005000067006F0044006F007800200045005A002B
:10051000000016034500720067006F0044006F0082
:100520007800200045005A00000011241FBECFEFC4
:10053000DAE0DEBFCDBF04B603FE24C08091CE0159
:100540009091CF01A091D001B091D1018750904BF3
:10055000A740B04BB9F41092CE011092CF01109287
:10056000D0011092D10114BE84B7877F84BF88E187
:100570000FB6F89480936000109260000FBEE0E028
:10058000FFE3099511E0A0E0B1E0EAEAF7E402C078
:1005900005900D92A631B107D9F711E0A6E1B1E0BF
:1005A00001C01D92AE3CB107E1F70E940B090C940B
:1005B000D3230C940000FC01613109F464C0623162
:1005C000A8F46D3009F441C06E3040F46B3079F11D
:1005D0006C30A0F56A3009F084C022C06F3009F495
:1005E00041C08281603108F043C036C0653109F4F2
:1005F0005AC0663140F4633109F43FC082816431EE
:1006000008F04CC046C0673109F459C0673108F49E
:1006100050C0683109F459C0693109F062C05BC04B
:100620008281882309F45DC02FE533E05CC08281BC
:10063000882309F456C02EE333E055C08281882315
:1006400009F44FC021E233E04EC08281882309F4CF
:1006500048C028E033E047C0882309F442C023EFB4
:1006600032E041C082818823E1F122EE32E03BC0DA
:100670008823B9F125EC32E036C08281882389F1E4
:1006800020EB32E030C08281882359F12FE932E03B
:100690002AC0882331F126E832E025C0882309F1F9
:1006A0002DE632E020C08281882319F02CE532E06B
:1006B0001AC082818823A9F023E432E014C0828129
:1006C000882379F022E232E00EC08281882349F04B
:1006D00021E132E008C08281882319F020E032E075
:1006E00002C020E030E0C9010895089560919701AB
:1006F000709198018091990190919A010E94CC1A71
:1007000056985E9825982D9826982E9827982F9879
:10071000813019F0823031F403C0259A2D9A089562
:10072000269A2E9A089586E793E0009711F0FC012F
:10073000099580E090E0089556985E9825982D9848
:1007400026982E9827982F988FEF90E09093890005
:100750008093880090938B0080938A0090938D0003
:1007600080938C00259A2D9A84EF91E020E931E066
:10077000F9013197F1F70197D9F7269A2E9A84EF6C
:1007800091E020E931E0F9013197F1F70197D9F7CC
:10079000279A2F9A84EF91E020E931E0F90131970F
:1007A000F1F70197D9F725982D9884EF91E020E98A
:1007B00031E0F9013197F1F70197D9F726982E9892
:1007C00084EF91E020E931E0F9013197F1F70197E9
:1007D000D9F727982F9856985E9825982D9826989F
:1007E0002E9827982F98089589EA8093800089E0B1
:1007F0008093810024982C983F988AB18F748AB98D
:100800006E98479A8BB1806B8BB9769A0E949C0345
:1008100085E793E0009711F0FC01099580E090E0F6
:10082000089580E28093000180911601882371F47D
:100830000E94600481E08093160180E197E220E944
:1008400031E0F9013197F1F70197D9F780E40E947F
:10085000660480930001882371F50E9494048093BC
:100860000001882341F50E949404809300018823AD
:1008700011F58FE30E949404809300018823D9F43A
:100880000E948C0480E40E94660480930001882307
:1008900091F48CE00E94940480930001882359F421
:1008A0000E94940480930001882329F48FE30E941E
:1008B0009404809300010E948C04809100010895AB
:1008C0001092B9008AE08093B8000895982F84EAC6
:1008D0008093BC008091BC0087FFFCCF8091B90061
:1008E000887F883021F0803111F081E00895909365
:1008F000BB0084E88093BC008091BC0087FFFCCFE4
:100900009091B900987F983111F480E0089580E0CB
:10091000903409F081E0089584E98093BC008091CF
:10092000BC0084FDFCCF08958093BB0084E88093D5
:10093000BC008091BC0087FFFCCF8091B90090E0A3
:10094000887F883209F091E0892F089584E88093A8
:10095000BC008091BC0087FFFCCF8091BB00089554
:10096000E7E1F1E0E80FF11D80810895089580919D
:1009700000018823A9F480E40E94660480930001AA
:10098000882361F482E10E9494048093000188230B
:1009900029F48FEF0E949404809300010E948C043C
:1009A00084B1807F84B985B1807F85B98AB1837F26
:1009B0008AB98BB1837F8BB93E98469808950E947F
:1009C0001104809300010E94B70480B38C7080BB37
:1009D00081B3836F81BB80E090E0FC01E95EFE4F54
:1009E0001082FC01EB5DFE4F108201968E30910566
:1009F000A1F784EF93E0009711F0FC0109950895A9
:100A0000BF92CF92DF92EF92FF920F931F93CF93FB
:100A1000DF9380910001882379F0809133018F5F0B
:100A200080933301882341F40E94110480930001D4
:100A3000882311F40E949C0325E2E22E21E0F22E8D
:100A4000C0E0D0E090EAB92E81E0C82ED12C02E0BF
:100A5000C73010F580910001882309F045C080E47B
:100A60000E94660480930001882399F482E10E9429
:100A7000940480930001882361F4C6010C2E02C007
:100A8000880F991F0A94E2F780950E94940480933E
:100A900000010E948C0428C0CA30D9F0CB3040F449
:100AA000C83089F0C93090F4C73009F0A0C008C040
:100AB000CC30A1F0CC3080F0CD3009F098C011C01E
:100AC000209A289894C0219A299891C0229A2A980D
:100AD0008EC0239A2B988BC0529A01C0539A5B9870
:100AE00086C03E9A469883C080910001882311F009
:100AF00010E03EC080E40E946604809300018823D9
:100B000099F483E10E94940480930001882361F4A6
:100B100081E40E94660480930001882329F40E94E6
:100B2000A604182F109501C010E00E948C0420C06C
:100B300042E07C9902C034E001C030E07D9902C0FF
:100B400028E001C020E07E9902C090E101C090E061
:100B50008FB18095881F8827881F8295880F807E97
:100B6000152F1C251170142B132B122B192B182B3E
:100B7000F7018081811719F01083009301010E9411
:100B8000B70421960894E11CF11CCE30D10509F080
:100B90005FCF809101018823C9F0815080930101CA
:100BA000882329F080EA9FE00197F1F70FC020E049
:100BB00030E0F901E95EFE4FD901AB5DBE4F8C918B
:100BC00080832F5F3F4F2E30310599F783E993E003
:100BD000009711F0FC01099581E0DF91CF911F9101
:100BE0000F91FF90EF90DF90CF90BF9008958B2DE5
:100BF0008A95F1F75FB1799B9BCF40E09ACF08953A
:100C00009C018B3B910578F4883A910548F5853A2B
:100C10009105B8F48430910508F09FC081309105AA
:100C200009F099C095C0803E910508F494C0883EB3
:100C3000910508F492C0805F9040409708F08BC007
:100C400085C0853A910519F481E890E47DC0863A23
:100C5000910519F083E890E477C082E890E474C0CD
:100C6000883A910519F482EE94E46EC0893A9105B0
:100C700019F489EE94E468C08A3A910519F48AEE71
:100C800094E462C08B3A910519F485EB94E45CC05E
:100C90008C3A910519F486EB94E456C08D3A91058F
:100CA00019F487EB94E450C0803B910519F48CEC67
:100CB00094E44AC08E3A910519F48DEC94E444C052
:100CC0008F3A910519F483E895E43EC0813B910584
:100CD00019F48AE895E438C0823B910519F482E959
:100CE00095E432C0833B910519F484E995E42CC066
:100CF000843B910519F481E296E426C0853B910579
:100D000019F483E296E420C0863B910519F484E24D
:100D100096E41AC0873B910519F485E296E414C065
:100D2000883B910519F486E296E40EC0893B910553
:100D300019F487E296E408C08A3B910519F080E037
:100D400094E402C08AE296E49C0107C0306505C0C5
:100D500021E030E002C020E030E0C9010895E62F34
:100D6000F0E0EE0FFF1F9CE0799F90011124E20F4D
:100D7000F31F98EA899FC0011124E80FF91FE45579
:100D8000FF4F25913491C9010895FC01EE0FFF1F1B
:100D9000E458FF4F25913491C9010895FC01EE0FED
:100DA000FF1FE450FE4F25913491C90108950E9420
:100DB000AF06AC018050914080509F4118F4CA01A9
:100DC0009F710895CA01805090428050904128F44C
:100DD000CA019F700E94CE060895CA0180509043B8
:100DE0008050904120F4CA019070906C089580E585
:100DF0004030580771F40E94D21084EC99E020E949
:100E000031E0F9013197F1F70197D9F70E94E81B1A
:100E10000EC120E54130520731F48091AE0181606E
:100E20008093AE0104C1CA0180509045805090412A
:100E300008F056C0652F77276F70707061307105AC
:100E4000F9F49A01A4E0220F331FAA95E1F720706C
:100E50003370CA01F3E0880F991FFA95E1F78076A5
:100E60009070282B392B3C684370507002C0660F7D
:100E7000771F4A95E2F76F717070262B372B2EC0C3
:100E80006230710529F4942F8827816F906A089544
:100E90006330710551F49A0173E0220F331F7A9584
:100EA000E1F7207E37703C680CC06430710561F555
:100EB0009A0163E0220F331F6A95E1F7207E3770B5
:100EC0003A684370507081E090E002C0880F991F2B
:100ED0004A95E2F78F719070282B392BC90108953C
:100EE000CA01805090478050904120F4CA019F7001
:100EF00090620895CA01805090488050904120F43B
:100F0000CA019F70906A0895403E5105F0F4403C3C
:100F1000510588F54133510509F476C04233510536
:100F200048F44932510509F465C04A32510509F0C7
:100F30007AC06FC04933510511F142385105F9F0BB
:100F40004533510509F06FC050C0433E510569F16A
:100F5000443E510540F4403E5105C1F0423E51052A
:100F600009F061C01DC0463E510559F1473E51058B
:100F700009F059C02BC0CA010E94C506089580918E
:100F8000BF0180FD0AC081FD08C04DC08091BF0136
:100F900080FF03C089E390E047C080EE90E044C04A
:100FA0008091BF0182FD08C004C08091BF0182FF13
:100FB00003C082EE90E038C084FD11C083EE90E063
:100FC00033C08091BF0183FD08C004C08091BF0180
:100FD00083FF03C086EE90E027C084FF03C080E05B
:100FE00090E022C087EE90E01FC08091BF0185FF96
:100FF00005C007C08091BF0185FF03C085E390E075
:1010000013C089E290E010C08091BF0186FF05C047
:1010100007C08091BF0186FF03C081E390E004C058
:101020008AE290E001C0CA010E9400060895089576
:1010300008951092C401089508950895809135018E
:101040000895DF93CF9300D00F92CDB7DEB7AC01F8
:101050008091C501843029F583E08093E9002FEF6A
:1010600095ED05C0892F8A95F1F7222329F080910B
:10107000E800215085FFF6CF8091E80085FF11C080
:101080005B834A8383E08983CE01019663E070E04D
:1010900040E050E00E94840B8091E8008E778093BE
:1010A000E8000F900F900F90CF91DF910895DF939C
:1010B000CF9300D00F92CDB7DEB7AC018091C501C0
:1010C000843029F583E08093E9002FEF95ED05C08A
:1010D000892F8A95F1F7222329F08091E800215089
:1010E00085FFF6CF8091E80085FF11C05B834A83BE
:1010F00082E08983CE01019663E070E040E050E039
:101100000E94840B8091E8008E778093E8000F9016
:101110000F900F90CF91DF910895AC018091C501A0
:10112000843001F582E08093E9002FEF95ED05C052
:10113000892F8A95F1F7222329F08091E800215028
:1011400085FFF6CF8091E80085FF0CC0CA0165E0FD
:1011500070E040E050E00E94840B8091E8008E77C0
:101160008093E80008950F931F93182F092F9091F3
:10117000C501943009F04CC0809102018823E1F050
:1011800080910D018823C1F09093E9009FEF25E144
:1011900005C0822F8A95F1F7992329F08091E80004
:1011A000915085FFF6CF8091E80085FF31C0812FF7
:1011B000902F60E170E018C081E08093E9009FEF1C
:1011C00025ED05C0822F8A95F1F7992329F08091AA
:1011D000E800915085FFF6CF8091E80085FF18C0A8
:1011E000812F902F68E070E040E050E00E94840B77
:1011F0008091E8008E778093E800A6E3B1E0212F8C
:10120000302FC901FC0180E101900D928150E1F77E
:101210001F910F91089584B7877F84BF88E10FB62F
:10122000F89480936000109260000FBE80E090E020
:1012300020E80FB6F89420936100809361000FBE00
:101240000E94D00F0E94620C0E94C30C8091E200A9
:1012500084608093E20078940E94610F0E946C1079
:1012600083E091E00E94770F0CC00E94151B8091D3
:10127000C301882331F00E946D1B882311F00E9466
:10128000990A8091C501853081F30E94D60FF9CF6C
:101290008091C401882349F40E94620C0E94C30C0F
:1012A0008091E20084608093E20008958091C701FC
:1012B000833009F457C0843030F4813071F08230CB
:1012C00009F0B1C098C08A3009F485C08B3009F4A8
:1012D0006AC0893009F0A7C020C08091C601813A58
:1012E00009F0A1C08091E800877F8093E800809199
:1012F000CA019091CB01892B21F486E391E060E152
:1013000003C080E090E060E070E00E94AF0A80914E
:10131000E8008B778093E80008958091C6018132C0
:1013200009F081C08091CA019091CB01009719F01A
:10133000039709F078C08091E800877F8093E800E8
:1013400005C08091C501882309F46DC08091E80033
:1013500082FFF7CF8091F100809335018091E80002
:101360008B771CC08091C601813A09F05CC08091E6
:10137000CA019091CB01892B09F055C08091E800FA
:10138000877F8093E8008091E80080FFFCCF809108
:1013900002018093F1008091E8008E778093E8004D
:1013A0000E940F0C08958091C6018132E1F5809171
:1013B000CA019091CB01892BB1F58091E800877F1C
:1013C0008093E8000E940F0C8091C8018093020175
:1013D0000E94D21008958091C601813221F580913A
:1013E000E800877F8093E8000E940F0C8091C9017C
:1013F0008093340108958091C601813AA1F48091CF
:10140000E800877F8093E8008091E80080FFFCCFB0
:10141000809134018093F1008091E8008E77809371
:10142000E8000E940F0C089581E061EC42E00E9408
:10143000D70B82E061EC42E00E94D70B83E061ECC5
:1014400042E00E94D70B84E061EC42E10E94D70B9E
:1014500008950E94661B0895DA019330C1F094301C
:1014600030F4913051F0923009F05BC00BC09132F2
:1014700021F1923209F055C037C0E7E7F4E022E1EC
:1014800030E053C0E9E8F4E02DE630E04EC08130B2
:1014900051F0813020F0823009F043C008C0E6EFFF
:1014A000F4E0849107C0EAEFF4E0849103C0E2E144
:1014B000F5E08491282F30E038C0613051F0613080
:1014C00028F0623059F0633061F50BC0EBE9F4E0CD
:1014D00002C0E4EBF4E029E030E027C0EDECF4E0FA
:1014E000FACFE6EEF4E0F7CF613061F0613028F03A
:1014F000623069F06330A9F40FC0ECE7F3E02FE34A
:1015000030E013C0EBEBF3E02DE430E00EC0E8E098
:10151000F4E026E330E009C0EEE3F4E029E330E054
:1015200004C0E0E0F0E020E030E0ED93FC93C9017E
:10153000089580E189BD82E189BD09B400FEFDCF37
:101540008091D8008F7D8093D8008091E0008260E8
:101550008093E0008091E00081FDFCCF08959C0124
:101560004091CC015091CD014617570718F4F9016D
:1015700090E043C06115710511F0AB01F8CF809187
:10158000E8008E778093E80040E050E0F0CF809153
:10159000C501882309F447C0853009F446C080910D
:1015A000E80083FD44C08091E80082FD36C0809150
:1015B000E80080FF22C08091F3009091F200782F24
:1015C00060E0292F30E0262B372B07C081918093D4
:1015D000F100415050402F5F3F4F4115510519F028
:1015E0002830310598F390E02830310509F491E076
:1015F0008091E8008E778093E8004115510539F617
:10160000992329F60AC08091C501882361F08530AD
:1016100061F08091E80083FD0AC08091E80082FFBC
:10162000F2CF80E0089582E0089583E0089581E09C
:1016300008959C014091CC015091CD014617570768
:1016400018F4F90190E044C06115710511F0AB0187
:10165000F8CF8091E8008E778093E80040E050E07A
:10166000F0CF8091C501882309F448C0853009F482
:1016700047C08091E80083FD45C08091E80082FD6D
:1016800037C08091E80080FF23C08091F3009091E3
:10169000F200782F60E0292F30E0262B372B08C08E
:1016A00084918093F1003196415050402F5F3F4F1D
:1016B0004115510519F02830310590F390E028309C
:1016C000310509F491E08091E8008E778093E8007D
:1016D0004115510531F6992321F60AC08091C501C3
:1016E000882361F0853061F08091E80083FD0AC0B5
:1016F0008091E80082FFF2CF80E0089582E00895B3
:1017000083E0089581E00895BF92CF92DF92EF9237
:10171000FF920F931F93CF93DF93182F092F7B0115
:101720006A010E94300CB82E8823B1F5812F902FCA
:101730009C01E901C114D10439F0F6018081918145
:10174000E81AF90AC80FD91F00E010E022C0809102
:10175000E80085FD16C08091E8008E778093E80050
:10176000C114D10449F0F60180819181800F911F4D
:101770009183808385E011C00E94300C882349F05A
:101780000CC089918093F1000894E108F1080F5F83
:101790001F4FE114F104D9F68B2DDF91CF911F91EA
:1017A0000F91FF90EF90DF90CF90BF900895382F6A
:1017B000282F2EC0822F8F708093E900231721F4E9
:1017C000762F942F50E006C07091EC009091ED00C0
:1017D0005091F00091FF1BC08091EB008E7F8093B1
:1017E000EB008091ED008D7F8093ED008091EB0008
:1017F00081608093EB007093EC009093ED00509328
:10180000F0008091EE0087FD02C080E008952F5F18
:10181000273080F23F703093E90081E00895809195
:10182000C60188239CF404C08091C5018823B9F0C7
:101830008091E80082FFF8CF8091E8008B77809359
:10184000E80008958091C501882349F08091E8005F
:1018500080FFF8CF8091E8008E778093E8000895AC
:101860004091E4005091E50024E68091EC0080FF77
:1018700024C08091E80080FD1EC08091C5018823AE
:1018800011F482E00895853011F483E00895809189
:10189000EB0085FF02C081E008958091E400909103
:1018A000E5008417950709F3222311F484E00895D5
:1018B0002150AC01DACF80E008958091E80082FFEA
:1018C000DCCFF9CF0E94D50C0E94DD0CE0EEF0E0F9
:1018D000808181608083A8EDB0E08C918F778C93BC
:1018E00019BCE7EDF0E080818E7F80838C918F7E44
:1018F0008C931092C4010895EF92FF920F931F935F
:101900000E94D50C0E94DD0C08ED10E0F8018081EA
:101910008F77808380818068808380818F7D8083C2
:1019200019BC1092C5011092C1011092C30110920E
:10193000C20180EEE82EF12CF70180818B7F80833D
:10194000F80180818160808380E060E042E00E9455
:10195000D70BE1EEF0E080818E7F8083E2EEF0E055
:10196000808181608083808188608083F7018081AD
:101970008E7F8083F8018081806180831F910F9129
:10198000FF90EF900895E8EDF0E080818F7E8083F6
:10199000E7EDF0E080818160808384E082BF81E0B8
:1019A0008093C4010E947C0C0895E8EDF0E08081F2
:1019B0008E7F80831092E20008951092DA001092D8
:1019C000E10008951F920F920FB60F9211241F93FA
:1019D0002F933F934F935F936F937F938F939F9337
:1019E000AF93BF93EF93FF931091E9008091EC00C8
:1019F0001092E9008091F000877F8093F000789446
:101A00000E94F00D1092E9008091F00088608093B0
:101A1000F0001F701093E900FF91EF91BF91AF911B
:101A20009F918F917F916F915F914F913F912F91F6
:101A30001F910F900FBE0F901F9018951F920F923D
:101A40000FB60F9211242F933F934F935F936F9391
:101A50007F938F939F93AF93BF93EF93FF93809167
:101A6000E10082FF0BC08091E20082FF07C08091FD
:101A7000E1008B7F8093E1000E94600F8091DA008B
:101A800080FF1FC08091D80080FF1BC08091DA00CA
:101A90008E7F8093DA008091D90080FF0DC080E1B5
:101AA00089BD82E189BD09B400FEFDCF81E080934C
:101AB000C5010E94480905C019BC1092C5010E94C9
:101AC00019088091E10080FF19C08091E20080FF39
:101AD00015C08091E2008E7F8093E2008091E20049
:101AE00080618093E2008091D80080628093D8006A
:101AF00019BC85E08093C5010E941D088091E1001A
:101B000084FF30C08091E20084FF2CC080E189BD59
:101B100082E189BD09B400FEFDCF8091D8008F7DA0
:101B20008093D8008091E1008F7E8093E1008091C6
:101B3000E2008F7E8093E2008091E20081608093DA
:101B4000E2008091C101882311F084E007C08091F8
:101B5000E30087FD02C081E001C083E08093C501FE
:101B60000E94290A8091E10083FF29C08091E20050
:101B700083FF25C08091E100877F8093E10082E0B0
:101B80008093C5011092C1018091E1008E7F809306
:101B9000E1008091E2008E7F8093E2008091E2007C
:101BA00080618093E20080E060E042E00E94D70B19
:101BB0008091F00088608093F0000E941C08FF91E3
:101BC000EF91BF91AF919F918F917F916F915F91B5
:101BD0004F913F912F910F900FBE0F901F9018952E
:101BE0001F93DF93CF93CDB7DEB7AC970FB6F894C2
:101BF000DEBF0FBECDBFE6ECF1E08091F100819336
:101C000021E0EE3CF207C9F70E9456098091E800F6
:101C100083FF3EC18091C6013091C701353009F480
:101C200087C0363040F43130C9F1313070F0333094
:101C300009F02EC133C0383009F4F9C0393009F445
:101C400009C1363009F024C197C0803821F08238AC
:101C500009F01EC108C09091C2018091C301882380
:101C600099F0926011C08091CA018F708093E90051
:101C70008091EB0090E025E0969587952A95E1F715
:101C8000982F91701092E9008091E800877F8093EF
:101C9000E8009093F1001092F100D4C0882319F06D
:101CA000823009F0F5C090E08F719070009721F0BC
:101CB000029709F0EDC00CC08091C801813009F095
:101CC000E7C01092C301333069F58093C3012AC085
:101CD0008091C801882331F52091CA012F7009F441
:101CE000D7C02093E9008091EB0080FF1BC0333008
:101CF00021F48091EB00806213C08091EB00806141
:101D00008093EB0081E090E002C0880F991F2A9534
:101D1000E2F78093EA001092EA008091EB0088607D
:101D20008093EB001092E9008091E800877F8DC0DE
:101D3000882309F0ADC01091C8011F778091E3009E
:101D40008078812B8093E3008091E800877F8093E7
:101D5000E8000E940F0C8091E80080FFFCCF80918A
:101D6000E30080688093E300112311F482E001C056
:101D700083E08093C5018CC08058823008F088C011
:101D80008091C8019091C90123E08C3D920709F030
:101D900034C083E08C838AE28B837FB7F894DE01C2
:101DA00015966EE040E050E011E2E62FF0E010936F
:101DB0005700849140FF03C082958F706F5F8F70D2
:101DC000282F30E08A3018F0C901C79602C0C90137
:101DD000C0968D939D934F5F5F4F4431510529F716
:101DE0007FBF8091E800877F8093E800CE01039653
:101DF0006AE270E00E94AF0A14C06091CA01AE01AD
:101E00004F5F5F4F0E942C0ABC01009709F440C04D
:101E10008091E800877F8093E80089819A810E9401
:101E2000190B8091E8008B778093E80031C08038EF
:101E300079F58091E800877F8093E8008091C10167
:101E40008093F1008091E8008E778093E8000E94F3
:101E50000F0C1EC08823E1F49091C8019230C0F4A9
:101E60008091E800877F8093E8009093C1010E94F1
:101E70000F0C8091C101882331F48091E30087FD2C
:101E800002C081E001C084E08093C5010E94140A71
:101E90008091E80083FF0AC08091E800877F8093EB
:101EA000E8008091EB0080628093EB00AC960FB667
:101EB000F894DEBF0FBECDBFCF91DF911F91089583
:101EC00008951F938091C501882379F01091E9004E
:101ED0008091EC001092E9008091E80083FF02C03D
:101EE0000E94F00D1F701093E9001F9108959093C8
:101EF0004B0180934A010895E0914A01F0914B0112
:101F0000309711F480E008950190F081E02D09955B
:101F10000895E0914A01F0914B01309721F0028041
:101F2000F381E02D09950895E0914A01F0914B016C
:101F3000309721F00480F581E02D099508959C01EA
:101F400080914801909149012817390779F0309321
:101F5000490120934801E0914A01F0914B013097EB
:101F600029F00680F781E02DC901099508959C01AB
:101F700080914601909147012817390779F03093F5
:101F8000470120934601E0914A01F0914B013097BF
:101F900029F00084F185E02DC9010995089508957F
:101FA0000E94CF0F08950E9418080895BF92CF9203
:101FB000DF92EF92FF920F931F93DF93CF93CDB7F2
:101FC000DEB72A970FB6F894DEBF0FBECDBF0E94D2
:101FD0000005EE24FF24BE2C8E2D0E94B004C82ED6
:101FE000F701E35BFE4FD080D82609F43FC0809113
:101FF000AE0181FF02C00E94B60400E010E0ED2DAA
:10200000F0E0CF01002E02C0959587950A94E2F783
:1020100080FF27C00E948B1B0983BA826C2D70E061
:10202000002E02C0759567950A94E2F76170707092
:102030006B8381609D838C83402F5B2D782F8D81F6
:102040000E944114F701E35BFE4F81E090E0002E17
:1020500002C0880F991F0A94E2F720812827208365
:102060001DC00F5F1F4F0630110559F60894E11C83
:10207000F11C8EE0E816F10409F0ADCF0E948B1B35
:102080002FEF2E832F8318868160782F9A87898778
:102090004FEF5FEF60E08A850E9441140E94601F4D
:1020A00010914C010E947C0F181731F00E947C0F98
:1020B00080934C010E94D30F2A960FB6F894DEBF8E
:1020C0000FBECDBFCF91DF911F910F91FF90EF9089
:1020D000DF90CF90BF9008950E94821B0E94DF0482
:1020E0000E94481C0895DF93CF9300D000D00F9238
:1020F000CDB7DEB70F900F900F900F900F90CF914C
:10210000DF910895DF93CF9300D000D000D0CDB7FA
:10211000DEB726960FB6F894DEBF0FBECDBFCF91C7
:10212000DF9108950E94B818482F892F82958F70EB
:10213000282F30E02C3031054CF42A3031056CF476
:102140002250304022303105C0F407C02C30310518
:1021500051F02F30310589F406C0403E10F0403F69
:1021600061F481E008959F70892F90E023E09695B7
:1021700087952A95E1F78170089580E008950E947F
:102180008C1A0E94611A0E94A41A0E94491F0E9480
:10219000551F80E090E00E949F0F80E090E00E9439
:1021A000B70F08950E947C1A0E94BF1008958823DB
:1021B00021F00E94751A0E94A41A0895882321F024
:1021C0000E946F1A0E94A41A0895282F882309F4E8
:1021D0004EC0823859F40E947C0F81FF48C089E3C9
:1021E0000E94EF190E94A41A89E30CC0833869F495
:1021F0000E947C0F80FF3BC083E50E94EF190E9484
:10220000A41A83E50E942D1A1FC0843859F40E9435
:102210007C0F82FF2CC087E40E94EF190E94A41A51
:1022200087E4F0CF8450813A10F4822FEBCF822FD5
:10223000805E883060F4277081E090E001C0880FF4
:102240002A95EAF70E94751A0E94A41A0895822F0F
:10225000855A833028F480E090E00E949F0F089513
:10226000285A233120F480E090E00E94B70F0895AF
:102270001F93182F882309F4D0C0823859F40E9484
:102280007C0F81FDCAC089E30E94EF190E94A41A45
:1022900089E30CC0833879F40E947C0F80FDBDC0B7
:1022A00083E50E94EF190E94A41A83E50E942D1A6B
:1022B0000E94A41AB2C0843859F40E947C0F82FD97
:1022C000ACC087E40E94EF190E94A41A87E4EECF05
:1022D0008450813A50F4812F0E948A21882309F08A
:1022E0009CC0812F0E94EF19E3CF812F805E883040
:1022F00050F4177081E090E001C0880F1A95EAF75A
:102300000E946F1AD5CF812F855A8330A0F4153AD9
:1023100019F481E890E00CC0163A19F482E890E0D4
:1023200007C0173A19F080E090E002C083E890E01F
:102330000E949F0F72C0812F885A833108F06DC0B0
:10234000183A19F482EE90E066C0193A19F489EE51
:1023500090E061C01A3A19F48AEE90E05CC01B3A32
:1023600019F485EB90E057C01C3A19F486EB90E025
:1023700052C01B3B19F483EB90E04DC01C3B19F499
:1023800084EB90E048C01D3A19F487EB90E043C01D
:10239000103B19F48CEC90E03EC01E3A19F48DEC21
:1023A00090E039C01F3A19F483E891E034C0113B42
:1023B00019F48AE891E02FC0123B19F482E991E008
:1023C0002AC0133B19F484E991E025C0143B19F4A9
:1023D00081E292E020C0153B19F483E292E01BC039
:1023E000163B19F484E292E016C0173B19F485E21B
:1023F00092E011C0183B19F486E292E00CC0193B40
:1024000019F487E292E007C01A3B19F080E090E0EF
:1024100002C08AE292E00E94B70F1F910895AF9226
:10242000BF92CF92DF92EF92FF920F931F93DF93B1
:10243000CF93CDB7DEB72A970FB6F894DEBF0FBEA5
:10244000CDBF5C01DE011196FC0185E001900D928B
:102450008150E1F70B81F501F580F2944FE0F42211
:10246000DE011696FE01319685E001900D928150B5
:10247000E1F73E812F8189859A85892B09F4F0C186
:102480002F3F09F0C0C13F3F09F0BDC1E9C18D2D0B
:102490008F70222311F4182F03C0182F1295107F6C
:1024A000002349F0112309F488C1812F0E947F1A6B
:1024B0000E94A41A82C18C2D0E94E510112309F4F8
:1024C000CFC1812F0E94851A0E94A41AC9C18D2DE7
:1024D0008F70203211F4182F03C0182F1295107F1F
:1024E000CC2021F0F1E0CF1611F516C0002359F0F1
:1024F000FF2009F431C121E0F21609F02DC1812F2E
:102500000E948F1AADC1FF2021F081E0F81609F476
:10251000A7C10E94921A26C1002329F0E1E0EF151D
:1025200008F49EC119C1FF2009F09AC11BC1002304
:1025300021F0FF2009F410C140C1FF2009F412C1AD
:1025400047C18D2D86958695837090E0009721F088
:10255000019709F085C10AC0002319F0C6019370E4
:1025600002C080E090E00E949F0F7AC1002319F022
:10257000C601937002C080E090E00E94B70F70C166
:10258000002321F08C2D0E94571E03C08C2D0E9429
:10259000C11E0E94551F64C18D2D837009F05EC05D
:1025A000002309F05DC12C2D229526952770220F5E
:1025B000220F8C2D8F70E82EFF2400E010E0022EF9
:1025C00004C0EE0CFF1C001F111F0A94D2F7C4FCBC
:1025D00005C060E070E080E090E00FC06FE070E068
:1025E00080E090E004C0660F771F881F991F2A952E
:1025F000D2F76095709580959095D694D694F3E037
:10260000DF224D2D50E041305105A9F042305105F7
:102610001CF4452B49F024C14230510589F0433068
:10262000510509F01DC113C06E297F29802B912B04
:102630000E94CA1915C16E297F29802B912B0BC0CE
:102640006E297F29802B912B0E94B91909C10E9404
:10265000CA19C801B7010E94DB1902C190E000232A
:1026600011F496958795817009F4FAC02C2D229566
:1026700026952770220F220F8C2D8F70E82EFF24B5
:1026800000E010E0022E04C0EE0CFF1C001F111F22
:102690000A94D2F7C4FC05C060E070E080E090E0EE
:1026A0000FC06FE070E080E090E004C0660F771F1D
:1026B000881F991F2A95D2F76095709580959095FF
:1026C000D694D69423E0D2224D2D50E041305105CE
:1026D000A9F0423051051CF4452B49F0C1C04230ED
:1026E000510589F04330510509F0BAC013C06E2975
:1026F0007F29802B912B0E941D19B2C06E297F2942
:10270000802B912B0BC06E297F29802B912B0E944F
:102710000C19A6C00E941D19C801B7010E942E19EC
:102720009FC080EFC81611F18C1528F0E0EECE1690
:1027300008F43FC009C0F2EFCF1661F1CF1628F1BF
:1027400023EFC216B1F52BC01C2D1F708D2D8F717C
:10275000002331F00E947B19812F0E94DE1080C07F
:102760000E945B19812F0E94D7107AC0002321F0AC
:10277000FF2009F075C004C081E08F1508F470C017
:102780008D2D8F710E943F196BC08D2D8F7100238D
:1027900029F119C08D2D8F710023A9F01FC00023CE
:1027A00029F08D2D8F710E9497195AC00E94A71988
:1027B00057C0002359F0FF2021F08C2D0E943811C2
:1027C0004FC08D2D8F710E947B194AC0FF2021F0D0
:1027D0008C2D0E94E51044C08D2D8F710E945B19D5
:1027E0003FC0EFE0DE22C5016C2D4D2D0E94DB02C3
:1027F0000E943D1835C0FFE0DF22C5016C2D4D2D34
:102800000E94FF052DC089819A810E94B8186C0131
:102810000E94B7180E94B6188D2D82958F7090E097
:102820008530910509F4ACCE8630910554F484309E
:1028300091050CF086CE2D2D207F02970CF047CE0F
:1028400026CE8C3091053CF48A3091050CF069CF8E
:10285000089731F4A1CE8C30910519F20F9759F2F7
:102860002A960FB6F894DEBF0FBECDBFCF91DF9191
:102870001F910F91FF90EF90DF90CF90BF90AF909E
:102880000895DF93CF93CDB7DEB72B970FB6F894AB
:10289000DEBF0FBECDBF342F4F83252F58876987EA
:1028A0007A878B87472F582FFE01319686E0DF010C
:1028B0001D928A95E9F76B8339832A834C835D8364
:1028C000432F522F8D819E810E947E172B960FB62B
:1028D000F894DEBF0FBECDBFCF91DF9108950F9367
:1028E0001F930091620115C010E0F801EE0FFF1F69
:1028F000E00FF11FEE0FFF1FED59FE4F4081518198
:1029000062817381848195810E9482100F5F1F4FC5
:10291000077080916101081739F71F910F91089591
:1029200040915B0150915C0160915D0170915E018D
:1029300080915F01909160010E94821008950F9331
:102940001F93CF93DF938091600182958F7009F080
:102950006DC080915D01882309F468C060916201B7
:102960000091610140915E0150915F0110915C0105
:1029700070915B01EA01C095D09555C04115510594
:1029800009F44FC01F3F49F480E090E07F3F11F40D
:1029900081E090E0882309F044C0262F30E0F9015F
:1029A000EE0FFF1FE20FF31FDF01AA0FBB1FAD5990
:1029B000BE4F11968C911197181799F58C91781735
:1029C00081F5EE0FFF1FEB59FE4F8081882349F5FB
:1029D00013968D919C9114978417950718F0841B7A
:1029E000950B02C08C0F9D1F883C9105D0F48091FF
:1029F00060018F70806180936001F901EE0FFF1F0D
:102A0000E20FF31FEE0FFF1FE859FE4F80818F701A
:102A1000806180838BE591E00E940F120E946F1409
:102A200005C06F5F6770601709F0A8CFDF91CF9185
:102A30001F910F910895DF92EF92FF920F931F93D2
:102A4000DF93CF93CDB7DEB76B970FB6F894DEBFA9
:102A50000FBECDBF8C01DC011296DC9012974C9119
:102A600011965C9111971396ED90FC90149720911C
:102A70005E0130915F0160915C0170915B012115F5
:102A8000310509F4DBC16F3F09F003C27F3F09F054
:102A900000C2D4C1E216F30640F0C701821B930BBB
:102AA000883C910508F0EEC008C0209530952E0DA9
:102AB0003F1D283C310508F0E5C080916001807F12
:102AC00009F095C06F3F09F0EAC17F3F09F0E7C107
:102AD00015C0741799F4DD2089F4809160018F701E
:102AE0008061809360010E9490148BE591E00E94C8
:102AF0000F1280916001F8018583BCC1FD82EC82D8
:102B00005A834983DB82DE011696FE01319685E009
:102B100001900D928150E1F76885DE011B96FE0160
:102B2000369685E001900D928150E1F72C853B852A
:102B30008E859F85892B09F451C02F3F09F0B3C1C1
:102B40003F3F09F0B0C14AC0FD82EC825A834983FD
:102B5000DB82DE011B96FE01319685E001900D922D
:102B60008150E1F7FC847B856D85809162019091B5
:102B700061011FC0282F30E0F901EE0FFF1FE20FA7
:102B8000F31FDF01AA0FBB1FAD59BE4F11968C91E9
:102B90001197F81651F48C91781739F4EE0FFF1F46
:102BA000EB59FE4F80816817C9F42F5F3F4F822F8A
:102BB00087708917F9F68DC19F7059F0442349F445
:102BC00059C19F7031F0D80115968C91807F09F41E
:102BD00051C1405E483008F44DC148C1DD2009F4C0
:102BE00049C18091600181608093600143C16F3F62
:102BF00009F05DC17F3F09F05AC114C0741791F408
:102C0000DD2081F480916001F8018583C8010E9474
:102C10000F12ABE5B1E0F80186E001900D92815012
:102C2000E1F720C15A83498389819A810E949210D9
:102C3000882309F41BC1DD2009F418C1309160011B
:102C4000832F82958F7090E002979CF090915C01A9
:102C500020915B01FE01709686E0DF011D928A954E
:102C6000E9F7998B288BFC8AEB8A3D8BCF010E9478
:102C70000F12ABE5B1E0F80186E001900D928150B2
:102C8000E1F7EEC080916001807FA9F47E2DFD8286
:102C9000EC825A834983DB826D2D8D810E947310F3
:102CA0000BE511E0C8010E940F1286E0F8011192B5
:102CB0008A95E9F7C0C06F3F09F0FDC07F3F09F07A
:102CC000FAC014C0741791F4DD2081F48091600182
:102CD000D80115968C93C8010E940F12EBE5F1E024
:102CE00086E0DF011D928A95E9F7BEC05A834983C9
:102CF00089819A810E949210882309F4B7C0DD204F
:102D000009F4B4C030916001832F82958F7090E0F8
:102D100002979CF090915C0120915B01FE017696F8
:102D200086E0DF011D928A95E9F79F8B2E8BFA8E44
:102D3000E98E3B8FCF010E940F12ABE5B1E0F801A5
:102D400086E001900D928150E1F78AC06F3F09F053
:102D5000B6C07F3F09F0B3C071C0E216F30640F081
:102D6000C701821B930B883C910508F053C008C033
:102D7000209530952E0D3F1D283C310508F04AC0A6
:102D8000DD2009F473C06F3F09F09FC07F3F09F059
:102D90009CC029C0741739F59091600190FD1AC04C
:102DA000892F82958F70B1F0F80195838F3031F0C3
:102DB0008F5F8295807F9F70982B9583C8010E94BA
:102DC0000F12ABE5B1E0F80186E001900D92815061
:102DD000E1F748C0ABE5B1E0F80186E001900D9263
:102DE0008150E1F741C05A83498389819A810E94C9
:102DF0009210882349F0ABE5B1E0F80186E001903C
:102E00000D928150E1F72CC0809160018160809328
:102E100060012CC07E2DFD82EC825A834983DB82C7
:102E20006D2D8D810E947310EBE5F1E086E0DF01EE
:102E30001D928A95E9F70E9490141CC0DD20B1F024
:102E40005A83498389819A810E949210882371F064
:102E5000ABE5B1E0F80186E001900D928150E1F719
:102E60000E949F140E94901481E005C0C8010E9436
:102E70000F12FACF80E06B960FB6F894DEBF0FBE4C
:102E8000CDBFCF91DF911F910F91FF90EF90DF9019
:102E9000089580915D01882309F458CFFBCD651713
:102EA00009F02CCE16CE613009F498CE4DCE6517C0
:102EB00009F0B8CEA3CE651709F018CF03CF8091E3
:102EC0005D01882309F0BACF48CF651709F08BCF91
:102ED00061CF5A83498389819A810E94B818482F0B
:102EE000892F82958F70282F30E0223031050CF425
:102EF00063CE243031050CF0B9CF63CE0F931F930E
:102F0000DF93CF93CDB7DEB72C970FB6F894DEBF23
:102F10000FBECDBF4F83588769877A878B879C8781
:102F20008E01095F1F4FC8010E941B158823D9F02D
:102F300028853F818A859B85892B09F46BC02F3FAB
:102F400049F480E090E03F3F11F481E090E0882375
:102F500009F060C04F81588569857A858B859C858D
:102F60000E94821057C0DE011196F80186E00190A0
:102F70000D928150E1F7F981EA814C815D81411523
:102F8000510509F447C0EF3F09F04CC0FF3F09F07D
:102F900049C040C0F983EA835D834C83F901EE0F99
:102FA000FF1FE20FF31FEE0FFF1FED59FE4FDE0173
:102FB000119686E00D9001928150E1F760936101D6
:102FC0000E946F1427C0919FC00111248D599E4FFC
:102FD0000E941B15882309F445C08091620190E08E
:102FE000FC01EE0FFF1FE80FF91FEE0FFF1FED5959
:102FF000FE4F4081518162817381848195810E945D
:1030000082108091620190E00196877090708093A9
:10301000620101C016E090916201809161019817F0
:1030200091F620C080916101282F30E02F5F3F4F43
:10303000B90167707070215030408091620190E05A
:103040006817790709F0A6CF0E94D210109261018B
:1030500010926201EBE5F1E086E0DF011D928A95B6
:10306000E9F7D8CF2C960FB6F894DEBF0FBECDBFD0
:10307000CF91DF911F910F910895CF92DF92EF9240
:10308000FF921F93CF93DF93EC01009709F466C082
:1030900010E090EAC92E9FE0D92E81E0E82EF12CB5
:1030A000FE0121969491943748F4943008F044C07E
:1030B000913079F0923009F051C01BC0953709F476
:1030C00037C0953750F1892F8458803708F046C0B3
:1030D00037C0FE0121969491892F805E883060F57B
:1030E00097708E2D01C0880F9A95EAF70E947F1A7B
:1030F0000FC0FE0121969491892F805E883058F48C
:1031000097708E2D01C0880F9A95EAF70E94851A54
:103110000E94A41A19C0892F15C0FE01249104C071
:10312000C6010197F1F721502223D1F721960CC057
:10313000FE012196149108C0892F0E94381104C005
:10314000892F8F770E94E510212F04C0C6010197B7
:10315000F1F72150222309F4A3CFF8CFDF91CF91CB
:103160001F91FF90EF90DF90CF90089508950895FC
:10317000CF92DF92EF92FF920F931F93CF93DF9343
:103180006C01E0909301F0909401009195011091F1
:1031900096018091970190919801A0919901B09129
:1031A0009A01E82AF92A0A2B1B2BCFE1D0E0D8019B
:1031B000C7010C2E04C0B695A795979587950A94DC
:1031C000D2F781709070892B41F08C2FB6010E944C
:1031D000D7069C018130910551F421978FEFCF3FA5
:1031E000D80729F780E0B6010E94D7069C01822FFC
:1031F000DF91CF911F910F91FF90EF90DF90CF90D3
:10320000089560939701709398018093990190932A
:103210009A010E94BF1008959B01AC016091970133
:10322000709198018091990190919A01622773277A
:10323000842795270E94011908959B01AC01609194
:103240009701709198018091990190919A01622360
:103250007323842395230E94011908959B01AC01D7
:1032600060919701709198018091990190919A01D4
:10327000622B732B842B952B0E940119089521E05A
:1032800030E040E050E004C0220F331F441F551FC0
:103290008A95D2F78091970190919801A091990118
:1032A000B0919A01282739274A275B27CA01B9011B
:1032B0000E940119089521E030E040E050E004C090
:1032C000220F331F441F551F8A95D2F72095309542
:1032D000409550958091970190919801A091990106
:1032E000B0919A01282339234A235B23CA01B901EB
:1032F0000E940119089521E030E040E050E004C050
:10330000220F331F441F551F8A95D2F780919701D2
:1033100090919801A0919901B0919A01282B392B95
:103320004A2B5B2BCA01B9010E940119089521E0C3
:1033300030E040E050E004C0220F331F441F551F0F
:103340008A95D2F7CA01B9010E940119089560E077
:1033500070E080E090E00E9401190895609393016D
:103360007093940180939501909396010E94BF10F1
:1033700008959B01AC01609193017091940180913B
:1033800095019091960162277327842795270E94C3
:10339000AE1908959B01AC01609193017091940165
:1033A0008091950190919601622373238423952344
:1033B0000E94AE1908959B01AC0160919301709138
:1033C00094018091950190919601622B732B842B2F
:1033D000952B0E94AE1908950E94AE190895382FBA
:1033E000809102018823E1F080910D018823C1F0D2
:1033F000832F8695869586958F3070F5E0910E0126
:10340000F0910F01E80FF11D377081E090E002C0EC
:10341000880F991F3A95E2F72181282B218308957F
:10342000A0910E01B0910F01FD0120E08FEF92817C
:10343000931791F08F3F19F4992309F4822F2F5F8E
:1034400031962E30A1F78F3F39F0992787FD90955F
:10345000A80FB91F12963C930895482F809102013E
:103460008823E9F080910D018823C9F0842F869587
:10347000869586958F3020F5E0910E01F0910F0131
:10348000E80FF11D477081E090E002C0880F991F9E
:103490004A95E2F78095218182238183089520E077
:1034A00030E0E0910E01F0910F01E20FF31F8281F5
:1034B000841709F412822F5F3F4F2E30310589F7B0
:1034C000089581E090E0E0910E01F0910F01E80F86
:1034D000F91F1082019680319105A9F70895909106
:1034E000AB01982B9093AB01089580959091AB011F
:1034F00098239093AB0108951092AB010895909199
:10350000AD01982B9093AD01089580959091AD01F8
:1035100098239093AD0108951092AD010895809382
:10352000AC0108951092AC010895E0910E01F09164
:103530000F0120E091E0818181112F5F9F5F319623
:103540009031C9F7822F0895E0910E01F0910F019B
:103550008091AB018083E0910E01F0910F01808199
:103560009091AD01892B80839091AC01992369F0F2
:10357000E0910E01F0910F018081892B80830E94E0
:10358000951A882311F00E94921A80910E01909151
:103590000F010E94890F08959B01AC01AA27BB2748
:1035A0000097A105B10521F4DA01C90160E001C06D
:1035B00060E1292F3A2F4B2F552721153105410561
:1035C000510519F49C01AD0101C0685FDA01C90120
:1035D00074E0B695A795979587957A95D1F700975A
:1035E000A105B10519F4DA01C90101C06C5F9C01A4
:1035F000AD01F2E05695479537952795FA95D1F7A5
:10360000211531054105510519F49C01AD0101C099
:103610006E5F5695479537952795211531054105DC
:10362000510509F06F5F862F08958091C5018430A0
:1036300009F11092AF0120E488E190E00FB6F89410
:10364000A895809360000FBE2093600083B7817FB0
:10365000846083BF83B7816083BF7894889583B784
:103660008E7F83BF88E10FB6F8948093600010923C
:1036700060000FBE0895089508951F920F920FB62F
:103680000F9211248F939F93AF93BF938091AF01BB
:10369000882399F48091B0019091B101A091B20179
:1036A000B091B3014196A11DB11D8093B0019093DB
:1036B000B101A093B201B093B301BF91AF919F91BB
:1036C0008F910F900FBE0F901F9018950E94D210EF
:1036D0000E947C0F0E94180808951F930E943B1BB4
:1036E0000E9400050E943C1B10E0812F0E94B00444
:1036F000882311F081E004C01F5F1E30B1F780E025
:103700001F91089582E084BD93E095BD9AEF97BD27
:1037100080936E0008958FB7F8942091B001309196
:10372000B1014091B2015091B3018FBFC901089519
:10373000EF92FF920F931F93BC018FB7F894E09024
:10374000B001F090B1010091B2011091B3018FBFAF
:10375000A801970140705070CB01A0E0B0E028179D
:1037600039074A075B0720F09701261B370B05C076
:103770009B01209530952E0D3F1DC9011F910F9182
:10378000FF90EF9008951F920F920FB60F921124A1
:103790008F939F93AF93BF938091B0019091B101AC
:1037A000A091B201B091B3010196A11DB11D80930A
:1037B000B0019093B101A093B201B093B301BF9156
:1037C000AF919F918F910F900FBE0F901F90189502
:1037D0000E94620CF89480E29EE420E931E0F90155
:1037E0003197F1F70197D9F787E090EBA7E0B0EBBD
:1037F0008093CE019093CF01A093D001B093D101DB
:103800002CE088E190E00FB6F894A89580936000D2
:103810000FBE20936000FFCFEF92FF920F931F9394
:10382000CF93DF93082F10E0812F0E94B004C0E0F7
:10383000D0E0E82EFF24C7010C2E02C09595879595
:103840000A94E2F780FF09C080E06C2F712F0E947C
:10385000AF06081711F481E008C02196C630D105E3
:1038600051F71F5F1E3001F780E0DF91CF911F916C
:103870000F91FF90EF9008951F93182F8CE20E94F4
:103880000C1C882319F0812F0E940C1C1F91089595
:103890001F93CF93DF930E94B61D882311F40E94DB
:1038A000C11D14E6C0E4DCE905C00E940005CE019C
:1038B0000197F1F71150C8F789E20E943C1C882358
:1038C00009F02FC18AE20E943C1C882311F00E945B
:1038D000C11D85E00E943C1C882311F00E94E81B5A
:1038E0000E94B11D8093AE0187E00E943C1C88239A
:1038F000B9F18BE10E943C1C882349F09091AE0104
:10390000892F869580958170880F9D7F26C08EE0D7
:103910000E943C1C882359F09091AE01892F869516
:10392000869580958170880F880F9B7F16C080E1F7
:103930000E943C1C9091AE01882359F0892F8695F6
:103940008695869580958170880F880F880F977F60
:1039500004C0892F809581709E7F982B9093AE0133
:103960008091AE010E94A11D0E94A71D8093BF01FE
:1039700080EE0E943C1C882349F08091BF01982F63
:10398000909591708E7F892B8093BF0189E30E946F
:103990003C1C882359F09091BF01892F8695809512
:1039A0008170880F9D7F982B9093BF0182EE0E94BB
:1039B0003C1C882369F09091BF01892F86958695DC
:1039C00080958170880F880F9B7F982B9093BF0103
:1039D00086EE0E943C1C882379F09091BF01892FCC
:1039E00086958695869580958170880F880F880FBB
:1039F000977F982B9093BF0183EE0E943C1C8823F5
:103A000069F09091BF01892F82958F7080958170A8
:103A10008295807F9F7E982B9093BF0185E30E94C3
:103A20003C1C882379F09091BF01892F829586955F
:103A30008770809581708295880F807E9F7D982BFE
:103A40009093BF0181E30E943C1C882389F09091F0
:103A5000BF01892F829586958695837080958170A8
:103A60008295880F880F807C9F7B982B9093BF0155
:103A700081E10E943C1C882379F08091BF01982F3E
:103A8000991F9927991F21E0922797959927979534
:103A90008F77892B8093BF018091BF010E94951D74
:103AA0008091BF01881F8827881F80930D0187E2BE
:103AB0000E943C1C182F8EE10E943C1C8111126058
:103AC0008FE10E943C1C8111146080E20E943C1C2A
:103AD0008111186081E20E943C1C8111106182E218
:103AE0000E943C1C8111106283E20E943C1C8111E7
:103AF000106484E20E943C1C81111068112341F083
:103B0000812F0E949B1D612F70E080E090E007C034
:103B10000E94AC1D90E0A0E0B0E0BC01CD010E948D
:103B2000EC19DF91CF911F910895682F84E090E008
:103B30000E94B0230895682F83E090E00E94B02394
:103B40000895682F82E090E00E94B023089584E0F9
:103B500090E00E94A223089583E090E00E94A223B7
:103B6000089582E090E00E94A223089580E090E012
:103B70000E94AA2320E08D5E9E4F09F421E0822F4F
:103B8000089580E090E06DEE7EEF0E94BE2382E01B
:103B900090E060E00E94B02383E090E060E00E944B
:103BA000B02384E090E060E00E94B02385E090E0E4
:103BB00060E00E94B02308958091BA0180FF0BC09D
:103BC0009091120185E0989FC001112495958795E9
:103BD0009595879530C081FF09C09091120185E0CD
:103BE000989FC00111249595879525C082FF03C039
:103BF000909112010DC08091B901882319F485E0DC
:103C000090E008956091130190911201861728F0B9
:103C100085E0989FC00111240EC0899F9001112456
:103C2000C901880F991F880F991F820F931F70E099
:103C30000E947B23CB018038910510F08FE7089517
:103C4000009709F481E008958091BA0180FF05C0D2
:103C5000809114018695869518C081FF04C08091DB
:103C60001401869512C082FF03C0809114010DC01B
:103C70002091B901222319F481E090E00895609128
:103C8000150180911401261710F090E007C0289FBD
:103C9000C001112470E00E947B23CB018038910584
:103CA00010F08FE70895009709F481E00895803FB0
:103CB00021F40E94DC1D819504C0813F29F40E94FB
:103CC000DC1D8093B6010895823F21F40E94DC1D23
:103CD000819504C0833F29F40E94DC1D8093B501C7
:103CE0000895893F19F40E94241E05C08A3F31F4CB
:103CF0000E94241E81958093B70108958B3F21F483
:103D00000E94241E819504C08C3F29F40E94241E29
:103D10008093B8010895843F21F48091B4018160BB
:103D200017C0853F21F48091B401826011C0863FA5
:103D300021F48091B40184600BC0873F21F480910D
:103D4000B401886005C0883F31F48091B40180617E
:103D50008093B40108958D3F21F48091BA01816070
:103D600005C08E3F31F48091BA0182608093BA0120
:103D700008958F3F29F48091BA0184608093BA013D
:103D80000895803F29F48091B60187FF6FC007C076
:103D9000813F41F48091B60118160CF067C0109273
:103DA000B60164C0823F29F48091B50187FF5EC0EF
:103DB00007C0833F41F48091B50118160CF056C03E
:103DC0001092B50153C0893F29F48091B7011816AC
:103DD0003CF04CC08A3F39F48091B70187FF46C060
:103DE0001092B70143C08B3F29F48091B80187FF3F
:103DF0003DC006C08C3F39F48091B8011816B4F567
:103E00001092B80133C0843F21F48091B4018E7FB9
:103E100005C0853F31F48091B4018D7F8093B4015A
:103E200025C0863F21F48091B4018B7FF7CF873F77
:103E300021F48091B401877FF1CF883F21F48091F4
:103E4000B4018F7EEBCF8D3F21F48091BA018E7F3C
:103E50000BC08E3F21F48091BA018D7F05C08F3F4A
:103E600029F48091BA018B7F8093BA018091B501CA
:103E7000882371F48091B601882351F48091B701B1
:103E8000882331F48091B801882311F41092B9018C
:103E90000895E4EBF1E085E0DF011D928A95E9F7F2
:103EA0001092B9011092BA01089584EB91E00E943A
:103EB000940F0E948B1B9093BC018093BB010895CB
:103EC0001F938091BB019091BC010E94981BAC0193
:103ED0002091B901222321F08091110190E006C0C8
:103EE000909110018AE0989FC0011124481759074A
:103EF00008F485C09091B501992369F48091B601C9
:103F0000882349F48091B701882329F48091B8016E
:103F1000882309F474C02F3F19F02F5F2093B90153
:103F2000191624F40E94DC1D8093B5018091B5011F
:103F300087FF05C00E94DC1D81958093B5018091AB
:103F4000B601181624F40E94DC1D8093B6018091FE
:103F5000B60187FF05C00E94DC1D81958093B601E4
:103F60006091B501662339F11091B601112319F161
:103F7000772767FD7095872F972F0E948C2223E368
:103F800033E343E35FE30E94F0220E9459226093EF
:103F9000B501612F772767FD7095872F972F0E94B6
:103FA0008C2223E333E343E35FE30E94F0220E9489
:103FB00059226093B6018091B701181624F40E942B
:103FC000241E8093B7018091B70187FF05C00E942E
:103FD000241E81958093B7018091B801181624F4AE
:103FE0000E94241E8093B8018091B80187FF05C00C
:103FF0000E94241E81958093B8010E94551F1F9135
:10400000089580E0089580E00895833099F1843028
:1040100030F4813069F0823009F06FC01AC0853009
:1040200009F44AC08530B8F1863009F066C055C041
:1040300020911001822F90E0860F911D8F3F9105F6
:1040400020F4260F2093100108958FEF8093100124
:10405000089520911101822F90E0860F911D8F3FCE
:10406000910520F4260F2093110108958FEF80937E
:104070001101089520911201822F90E0860F911D69
:104080008F3F910520F4260F2093120108958FEFA2
:1040900080931201089520911301822F90E0860FE2
:1040A000911D8F3F910520F4260F20931301089551
:1040B0008FEF80931301089520911401822F90E0D7
:1040C000860F911D8F3F910520F4260F2093140138
:1040D00008958FEF80931401089520911501822F88
:1040E00090E0860F911D8F3F910520F4260F2093BD
:1040F000150108958FEF809315010895833031F1F4
:10410000843030F4813061F0823009F04AC013C04D
:10411000853091F1853028F1863009F042C037C0F2
:1041200080911001681720F4861B80931001089578
:1041300010921001089580911101681720F4861BD8
:104140008093110108951092110108958091120138
:10415000681720F4861B80931201089510921201B3
:10416000089580911301681720F4861B8093130132
:10417000089510921301089580911401681720F496
:10418000861B809314010895109214010895809164
:104190001501681720F4861B80931501089510926D
:1041A0001501089521E030E040E050E004C0220F06
:1041B000331F441F551F8A95D2F7CA01B9010E94C7
:1041C000EC190E94D21008958B3109F463C08C3130
:1041D00000F58E3009F468C08F3068F4873009F438
:1041E00053C0883018F4863089F537C0883081F1A3
:1041F0008B3061F58DC0813109F478C0823118F4BB
:10420000803121F55DC0863109F482C08931F1F435
:104210007FC0853309F473C0863358F4873209F4BC
:104220006EC0883218F48E3188F06BC0893271F418
:1042300066C0833430F48A3308F065C0883331F4C3
:1042400067C0833409F45BC0883481F080E008954E
:104250000E94B11D0E94A71D59C08091AE01807FB0
:104260008093AE0181E08093BD0108950E94D21039
:1042700080E197E220E931E0F9013197F1F7019708
:10428000D9F70E94E81B42C08091AE0180FF2AC08E
:10429000807F29C08091AE01982F9695909591705E
:1042A000292F220F8D7F19C08091AE01982F9695EE
:1042B000969590959170292F220F220F8B7F0DC01C
:1042C0008091AE01982F96959695969590959170C0
:1042D000292F220F220F220F877F822B8093AE017E
:1042E0009923B1F081608093AE0110C00E94D2107A
:1042F00080910D0191E0892780930D0107C080E036
:1043000003C08D5101C089530E94D22081E00895DD
:1043100081E008951F93182F8091BD01813089F0AD
:10432000813020F0823009F0BFC03BC0E0910E0127
:10433000F0910F01E081E13169F0E23209F0B6C09D
:1043400009C0E0910E01F0910F01E081E13111F01F
:10435000E23249F4812F0E9401208823F9F4812F51
:104360000E94E420A4C0812F0E9403208823B1F47E
:10437000143161F0153128F41B3081F0103141F413
:104380000AC0193219F0183319F408C01092BD018F
:1043900080E090E08CC082E08093BD0181E090E0FD
:1043A00086C0193201F11A3270F41431E1F015317E
:1043B00020F4173009F064C065C0812F8E5186301B
:1043C00008F05EC01BC01E3409F455C01F3420F431
:1043D0001B3409F055C049C0113509F442C01235EB
:1043E00009F04EC03AC08091BE01882319F01092A6
:1043F000BE0146C081E08093BD0159C01232F9F080
:10440000133260F41F3199F0103218F41E3109F59F
:1044100010C0103281F01132E1F40FC0143299F063
:10442000143278F0153289F0163299F410C082E017
:1044300011C081E00FC083E00DC084E00BC085E0B7
:1044400009C086E007C087E005C088E003C089E0B6
:1044500001C080E08093BE0113C08091BE0161E085
:1044600007C08091BE0161E009C08091BE016AE091
:104470000E94052005C08091BE016AE00E947E2056
:1044800081E015C09AE09093100184E180931101BE
:1044900083E0809312019093130188E080931401CC
:1044A00088E280931501ECCF1092BD0180E01F914E
:1044B000089504D06894B1118DC0089570D088F02B
:1044C0009F5790F0B92F9927B751A0F0D1F0660F00
:1044D000771F881F991F1AF0BA95C9F712C0B1301B
:1044E00081F077D0B1E0089574C0672F782F8827C6
:1044F000B85F39F0B93FCCF3869577956795B3955A
:10450000D9F73EF490958095709561957F4F8F4FC8
:104510009F4F0895E89409C097FB3EF490958095CD
:10452000709561957F4F8F4F9F4F9923A9F0F92F79
:1045300096E9BB279395F695879577956795B795F7
:10454000F111F8CFFAF4BB0F11F460FF1BC06F5FDD
:104550007F4F8F4F9F4F16C0882311F096E911C0EF
:10456000772321F09EE8872F762F05C0662371F010
:1045700096E8862F70E060E02AF09A95660F771F24
:10458000881FDAF7880F9695879597F9089557FD54
:104590009058440F551F59F05F3F71F04795880FB1
:1045A00097FB991F61F09F3F79F087950895121648
:1045B00013061406551FF2CF4695F1DF08C01616F4
:1045C00017061806991FF1CF8695710561050894A5
:1045D0000895E894BB2766277727CB0197F90895BC
:1045E0000BD078C069D028F06ED018F0952309F070
:1045F0005AC05FC01124EECFCADFA0F3959FD1F35C
:10460000950F50E0551F629FF001729FBB27F00D80
:10461000B11D639FAA27F00DB11DAA1F649F6627D5
:10462000B00DA11D661F829F2227B00DA11D621F24
:10463000739FB00DA11D621F839FA00D611D221FDE
:10464000749F3327A00D611D231F849F600D211DC2
:10465000822F762F6A2F11249F5750408AF0E1F065
:1046600088234AF0EE0FFF1FBB1F661F771F881FAE
:1046700091505040A9F79E3F510570F014C0AACF49
:104680005F3FECF3983EDCF3869577956795B79599
:10469000F795E7959F5FC1F7FE2B880F911D9695C3
:1046A000879597F9089597F99F6780E870E060E033
:1046B00008959FEF80EC089500240A9416161706BB
:1046C00018060906089500240A9412161306140603
:1046D00005060895092E0394000C11F4882352F066
:1046E000BB0F40F4BF2B11F460FF04C06F5F7F4F1E
:1046F0008F4F9F4F089597FB092E07260AD077FD0D
:1047000004D00CD006D000201AF4709561957F4F2C
:104710000895F6F7909581959F4F0895AA1BBB1BAE
:1047200051E107C0AA1FBB1FA617B70710F0A61BB1
:10473000B70B881F991F5A95A9F780959095BC01D2
:10474000CD010895F999FECF92BD81BDF89A9927C0
:1047500080B50895A8E1B0E042E050E00C94C52394
:10476000262FF999FECF1FBA92BD81BD20BD0FB68D
:10477000F894FA9AF99A0FBE019608950E94B02310
:10478000272F0C94B123DC01CB01FC01F999FECF5A
:1047900006C0F2BDE1BDF89A319600B40D924150C9
:0A47A0005040B8F70895F894FFCFD9
:1047AA002002011E08B3088D0857082108019B0141
:0647BA000A14030A08289E
:00000001FF
